:04000000BE012C29E8
:10000800080064008C1E05281A0803142729BE1648
:10001800BE1EBE12BE191428BE154D2003183B285B
:100028000830A9006120A80DA90B1628BE1E46207D
:100038006B206720BE1A3B20402028080310272980
:10004800BE16BE1EBE123E192E28FE39BF003E1532
:10005800031027293E1A3628AC003E164D200318F7
:100068003B282C08542003183B28BE1E272946206D
:100078006B203E113E12BE114C0884004A088417BA
:1000880080044C284C0884004A09800584178005A0
:10009800080040206B20462067203F08BE19013821
:1000A800A8000830A900A80D03184020031C46200A
:1000B8006B206720A90B572840206B204C08840030
:1000C8004A080005FF3E4D0884004B0949284D08A1
:1000D80084004B0843280830AC004D0884004B08C6
:1000E8003F1999203F1D9B204C0884004A099F20F6
:1000F8002C08031927293F18BF204C088400A70C97
:10010800A60C00084A04031C4A0680008E20AC0B8B
:10011800812827294D0884004B0880060000942870
:100128009528962897288006080080049E28FF3A7C
:1001380080059F28FF3A841780052729A901A80070
:10014800FF30A807031CA907031C27290330A700B1
:10015800E630B020A428A701FC3EA600A709031C8E
:10016800BB28FF300000A6070318B628A6076400BE
:10017800A70FB5280800A801A901C628A70CA60C36
:10018800A80DA90DFF3E0318C2282908A7002808B2
:10019800A6002729A701A901A8000230DE28A70187
:1001A800A901A8000130DE28A8000630DE28A80032
:1001B8000430DE28AE0029082702031DE528280898
:1001C8002602043003180130031902302E05031DDE
:1001D800FF3027290038031DFF300405031DFF30B9
:1001E8002729AB01AA011030AC00270DAA0DAB0DD1
:1001F8002808AA022908031C290FAB0203180B2997
:100208002808AA0729080318290FAB070310A60D09
:10021800A70DAC0BF928260827291030AE00A70136
:10022800A601AD0CAC0C031C1F292808A607290839
:100238000318290FA707A70CA60CAB0CAA0CAE0B2A
:1002480015292A0827298313031383126400080039
:10025800831620309900203098008312903098003F
:100268008A110A1237298316031788018901031393
:10027800E03085008601C03087008801890183123B
:1002880085018601870188018901831685308100EF
:100298008B1783128A110A1256298B1B08008A11A0
:1002A8000A129E2D8A015121A0308B008A0151210A
:1002B800CE018A015121CF018A015121D0018A0141
:1002C8005121D1018A015121D2018A015121D30141
:1002D8008A015121D4018A015121D5018A01512174
:1002E800D6018A015121D7018A015121D8018A01F9
:1002F8005121D9018A015121DA018A015121DB01F9
:100308008A015121DC018A015121DD018A01512133
:10031800DE018A015121DF018A015121E0018A01B0
:100328005121E1018A015121E2018A015121E301B0
:100338008A015121E4018A015121E5018A015121F3
:10034800E6018A015121E7018A015121C7018A0189
:1003580051210230BB008A0151210130BA008A01C3
:1003680051210730CC000230CA000730CD000130DF
:10037800CB00A0308A01262000308A0126200030D8
:100388008A0124208A0151210730CC000230CA009A
:100398000730CD000130CB00A1308A0126208A0128
:1003A8000D20B9008A010D20C1008A010D20BC0072
:1003B8008A010B20BD008A0151213C08AC00AD0127
:1003C800A8010130A9008A011121ED002B08EE00D7
:1003D8003D086D07A2006E080318013EA3008A01BC
:1003E80051212208A0002308A1008A0151210130CF
:1003F800B8008A015121A401A5018A0151214810A0
:100408008A015121C8108A01512164008A110A12F7
:10041800C818702C8A0151212008A6002108A700BD
:10042800A8010130A9008A01F520BC008A015121E8
:100438002008A6002108A700A8010130A9008A0108
:10044800F5202A08BD008A0151210730CC0002306E
:10045800CA000730CD000130CB00A0308A01262029
:100468003C088A0126203D088A0124208A0151215E
:100478000730CC000230CA000730CD000130CB0075
:10048800A1308A0126208A010D20CE008A010D2084
:10049800CF008A010D20D0008A010D20D1008A01E9
:1004A8000D20D2008A010D20D3008A010D20D4002E
:1004B8008A010D20D5008A010D20D6008A010D2061
:1004C800D7008A010D20D8008A010D20D9008A01A1
:1004D8000D20DA008A010D20DB008A010D20DC00E6
:1004E8008A010D20DD008A010D20DE008A010D2021
:1004F800DF008A010D20E0008A010D20E1008A0159
:100508000D20E2008A010D20E3008A010D20E4009D
:100518008A010D20E5008A010B20E6008A0151219D
:100528002030A0070318A10A8A015121FF30410792
:10053800ED00FF300318013EEE006D08AC006E08B8
:10054800AD002030A800A9018A011121ED002B0877
:10055800EE002208ED0723080318013EEE072008E5
:10056800A6002108A7006E08A9006D088A01D820F6
:100578008A110A12031DC12ABA0A8A0151213A08AE
:10058800A6003B088A01D320ED000030481801304E
:10059800A60001308A01CE20EF006D0884006F08A4
:1005A8008A01EE208A110A12031D4E2B8A0151215D
:1005B800FF304107ED00FF300318013EEE006D08E3
:1005C800AC006E08AD002030A800A9018A011121F5
:1005D800ED002B08EE002208ED0723080318013E62
:1005E800EE072008A6002108A7006E08A9006D08DC
:1005F8008A01D8208A110A12031D062B2208A0009E
:100608002308A1008A01512164008A110A12851E5B
:10061800232B8A0151212408A6002508A700A90137
:1006280028308A01DB208A110A12031D062B8A0151
:100638005121A401A5018A0151218A01072A8A01B1
:1006480051212408A6002508A7000230A9008A30F5
:100658008A01D5208A110A12031DD02B8A01512143
:1006680064008A110A12851E232B8A015121481021
:100678008A0151212408A6002508A700A901643091
:100688008A01DB208A110A12031D392B8A015121A4
:10069800A401A5018A0151210130BA008A01512122
:1006A800B80A8A0151216400380839028A110A12ED
:1006B80003186B2B8A0151210130B8008A0151219E
:1006C8000130BD008A0151218A110A12842B8A0146
:1006D8005121FF303807ED00FF300318013EEE00CE
:1006E8006D08AC006E08AD000330A800A9018A01AE
:1006F8001121ED002B08EE006D0ABD008A01512181
:100708008A0151210730CC000230CA000730CD00E1
:100718000130CB00A0308A01262000308A01262033
:100728003D088A0124208A01512132308A01A22001
:100738008A0151210730CC000230CA000730CD00B1
:100748000130CB00A1308A0126208A010D20C1008A
:100758008A010D20BC008A010B20BD008A015121AD
:100768003C08AC00AD01A8010130A9008A011121A3
:10077800ED002B08EE003D086D07A2006E08031877
:10078800013EA3008A0151212208A0002308A100EC
:100798008A0151218A01072A8A01512148148A01B4
:1007A80051210130BA008A0151210F30CE008A014F
:1007B80051211430CF008A0151211430D0008A0110
:1007C80051211430D1008A0151210F30D2008A0101
:1007D80051212408A6002508A7000430A9004C30A0
:1007E8008A01D5208A110A12031D092C8A01512178
:1007F80064008A110A12851ED02B8A015121A40196
:10080800A5018A0151218A01072A8A01512148102C
:100818008A015121A401A5018A015121C8148A0124
:1008280051211F30CE008A0151210130CF008A01A9
:1008380051211F30D0008A0151210130D1008A0195
:1008480051211F30D2008A015121D3018A0151213F
:10085800D4018A015121D5018A015121D6018A0189
:100868005121D7018A015121D8018A015121D90189
:100878008A015121DA018A015121DB018A015121C2
:10088800DC018A015121DD018A015121DE018A0141
:100898005121DF018A015121E0018A015121E10141
:1008A8008A015121E2018A015121E3018A01512182
:1008B800E4018A015121E5018A015121E6018A01F9
:1008C800512164008A110A12851E092C8A015121BE
:1008D80018128A01512118168A0151215D08E20077
:1008E8008A0151215E08E3008A0151215F08E40072
:1008F8008A0151216008E5008A0151216108E6005A
:100908008A0151215808DD008A0151215908DE0069
:100918008A0151215A08DF008A0151215B08E00051
:100928008A0151215C08E1008A0151215308D8004D
:100938008A0151215408D9008A0151215508DA0049
:100948008A0151215608DB008A0151215708DC0031
:100958008A0151214E08D3008A0151214F08D40041
:100968008A0151215008D5008A0151215108D60029
:100978008A0151215208D7008A0151216808063C92
:100988008A110A12031CDA2C8A110A12CF24D20007
:100998008A110A12DA2C04308A00680882070034A7
:1009A8000134033407340F341F341F348A015121B2
:1009B8006908063C8A110A12031CF42C8A110A12CF
:1009C800E924D1008A110A12F42C04308A0069083B
:1009D800820700340134033407340F341F341F34C2
:1009E8008A0151216A08063C8A110A12031C0E2D3D
:1009F8008A110A120325D0008A110A120E2D053019
:100A08008A006A08820700340134033407340F343B
:100A18001F341F348A0151216B08063C8A110A12BF
:100A2800031C282D8A110A121D25CF008A110A12CB
:100A3800282D05308A006B088207003401340334FE
:100A480007340F341F341F348A0151216C08063CC7
:100A58008A110A12031C422D8A110A123725CE0068
:100A68008A110A12422D05308A006C088207003468
:100A78000134033407340F341F341F348A015121E1
:100A880064008A110A12851EFD298A015121640019
:100A98008A110A128C1E422D8A0151218A010520D1
:100AA800C0008A01512164004008F03C8A110A12F2
:100AB800031D422D8A01512164008A110A128C1EDD
:100AC8005E2D8A0151218A010520E8008A01512101
:100AD80064008A110A128C1E6A2D8A0151218A012A
:100AE8000520E9008A01512164008A110A128C1E2E
:100AF800762D8A0151218A010520EA008A015121B7
:100B080064008A110A128C1E822D8A0151218A01E1
:100B18000520EB008A01512164008A110A128C1EFB
:100B28008E2D8A0151218A010520EC008A0151216C
:100B38008A01702CA40A0319A50A8A110A127426BC
:100B4800C70A6400053047028A110A12031CAD2D3A
:100B5800C7014708A700043C8A110A12031CCE2DBE
:100B6800A70D8A110A12C025A60027108A110A1299
:100B7800C0258A002608820005308A0027088207D7
:100B88000534CE340534E3340534F83406340D34F2
:100B9800063422344E08C2004F08C3005008C4006F
:100BA8005108C5005208C6008A110A1237261E309D
:100BB800E7008A110A128B268A110A12A22E5308FC
:100BC800C2005408C3005508C4005608C500570899
:100BD800C6008A110A1237261D30E7008A110A1248
:100BE8008B268A110A12A22E5808C2005908C3007F
:100BF8005A08C4005B08C5005C08C6008A110A12BE
:100C080037261B30E7008A110A128B268A110A122E
:100C1800A22E5D08C2005E08C3005F08C400600819
:100C2800C5006108C6008A110A1237261730E70086
:100C38008A110A128B268A110A12A22E6208C20091
:100C48006308C3006408C4006508C5006608C600D8
:100C58008A110A1237260F30E7008A110A128B26EA
:100C68008A110A12A22E460885004508AC00AD017B
:100C78000830A800A9018A01112186004308AC00A8
:100C8800AD010230A800A9018A0111218800441A87
:100C98000615441E0611C4198614C41D861044196D
:100CA8000614441D0610C4188817C41C8813441859
:100CB8000817441C0813421A8716421E8712C219C5
:100CC8000716C21D071242190814421D0810C2183F
:100CD8008715C21C871142180715421C0711080006
:100CE80009108316091009308312CC000430CA0099
:100CF8000930CD000230CB00BF011F30A600A7018C
:100D08008A016F200914831609108312080009103C
:100D18008316091009308312CC000430CA00093048
:100D2800CD000230CB00BF016708A600A7018A01E9
:100D38006F20091483160910831208000B1109008B
:02400E00D22FAF
:00000001FF
